:1000000012C02BC02AC029C028C027C026C025C0C6
:1000100024C023C022C021C020C01FC01EC01DC0DC
:100020001CC01BC01AC011241FBECFE5D4E0DEBF28
:10003000CDBF10E0A0E6B0E0E6EBF0E002C0059036
:100040000D92A036B107D9F710E0A0E6B0E001C0EC
:100050001D92A036B107E1F701C0D2CFCFE5D4E0C1
:10006000DEBFCDBF83E087BB60E031E0132FCFEF71
:10007000D0E0F32F662309F43127A0E0B0E0AE0111
:10008000461B5109E32FEF2774E0662319F0862FF2
:100090008150F1F738BB20E0A417B50734F42F5F87
:1000A000822F992784179507D4F3E8BB715077FF07
:0600B000ECCF6F5FDFCF13
:00000001FF
